:020000040800F2
:10100000B8490020D110000809440008A5200008B4
:1010100000000000000000000000000000000000D0
:101020000000000000000000000000000D56000855
:101030000000000000000000B5480008495B0008FF
:10104000E310000800000000E3100008E3100008AF
:10105000E3100008E3100008E3100008E3100008A4
:1010600000000000E310000825150008C515000861
:10107000E3100008E3100008E3100008000000007F
:10108000E3100008515C0008E3100008E3100008BA
:10109000E3100008E3100008E3100008E310000864
:1010A000E3100008F1550008E3100008695C00082F
:1010B000E55C0008395D00080348854600F0D6F875
:1010C00000480047F9680008B84900200844F04784
:1010D0000448804704480047FEE7FEE7FEE7FEE7D6
:1010E000FEE7FEE7F55B0008B910000830B50B46D7
:1010F000014600202022012409E00D46D5409D42F2
:1011000005D31D469540491B254695404019154677
:10111000521E002DF1DC30BD70B50024254600289C
:1011200001DA01244042002901DA01254942FFF792
:10113000DDFFAC4200D04042002C00D0494270BDDF
:10114000F8B500242546002904DA0E4601240021C2
:101150004042B141002B04DA1E46002352420125D1
:10116000B34100F052F88C4617461E46AC4203D0FD
:10117000002540428D41AC46002C02D0002657424B
:101180009E4161463A46334601B0F0BD10B5202A73
:1011900004DB0846203AD040002110BD0B46D34066
:1011A000D0402024A21A91400843194610BD03469E
:1011B0000B439B0703D009E008C9121F08C0042A8B
:1011C000FAD203E00B780370401C491C521EF9D27E
:1011D0007047D2B201E00270401C491EFBD270473A
:1011E0000022F6E710B513460A4604461946FFF7F3
:1011F000F0FF204610BD0321001D401E037812029F
:101200001A43491EF9D510467047F0B51FB406467B
:10121000002082B005464024019100901BE0019916
:1012200022460F463046FFF7B1FF049A059B801A0D
:10123000994110D310461946224600F029F8361A73
:101240008F410197224601200021009F00F020F8E5
:1012500038184D4100902046641E0028DFDC019BB9
:1012600000982946324607B0F0BD0000064C012523
:10127000064E05E0E36807CC2B430C3C984710343E
:10128000B442F7D3FFF71CFFF87A0008187B000878
:1012900010B5202A04DB0146203A9140002010BD01
:1012A000914020239C1A0346E3401943904010BD0F
:1012B00030B58C180278401C13071B0F01D103783E
:1012C000401C120906D10278401C03E005780D701D
:1012D000401C491C5B1EF9D101E00B70491C521ED9
:1012E000FBD1A142E6D3002030BD0000F0B52C4870
:1012F00081684907C90F50D1006C2A4D82B26B69D1
:101300000120DC07284E2949002C0AD08A82284B6C
:10131000284930469A4201D2012200E000220A60A8
:1013200031E0254F9E433C880CD0244E9E430DD087
:10133000234C9C431DD0234C9C431DD0224C9C43EA
:101340001DD020E0A01838801C481CE07888801848
:1013500082B27A802869401C2861082807DBE008EF
:101360004883D0088883002038807880286114481A
:1013700009E0CA83154806E00A84154803E04A8458
:10138000144A528B8A8442030549520B8A628A6846
:10139000114B1A40121D8A6068610020F0BD0000E8
:1013A00000240140C00000208000001C0017002025
:1013B000DC05000060010020480200200001002040
:1013C000000200240000014000000244000001C0AF
:1013D000000002C4A0F7FF1FE8FFFF7FF0B51E4F1B
:1013E00085B03D691D4C6D1C3D612668A468029462
:1013F00000966C4665800190218162810393386A72
:1014000001011748091800220B4610461C5CFF2CEE
:1014100004D1401C1028F9D3002A17D010226846A6
:1014200000F00CF9386AF861401C386200010121B3
:1014300049031030884201D900203862F868094910
:10144000401CF8604867002005B0F0BD10226846D7
:1014500004F02CFFE6E700003C01002020710008AA
:1014600000D0000880160020002911D08268521890
:1014700082604368934200DCD21A00238361C36810
:10148000934201D1012343618260026952180261D3
:1014900008467047F0B50020174D0127144B154C36
:1014A0007F03E86017E0625A144EB24212D1EA6834
:1014B0000919521CEA604A882E69B24205D92A618C
:1014C000E8614A686A61421C2A624988994201D2ED
:1014D0000B46A861401C0101B942E4D3286A00010F
:1014E0001030B84201D900202862E868F0BD000041
:1014F000FFC99A3B00D000083C010020AA5500001B
:1015000010B50421054800F0C9F8054800218161A3
:10151000C1610161C1600162084610BD00D00008D0
:101520003C01002070B5234DE86A401CE862224C63
:1015300020688006C00F11D02868296B40182860E9
:10154000296B28465830064600F058F82020606085
:10155000B06900280AD000202863687220688005DE
:10156000C00F02D001204002606070BD304600F024
:101570000BF912494A78A3585B085B00A350F36843
:1015800032684E78D2180C4B0C33F2500A4B4A7822
:101590001B1DD658360C36040643D650497862587F
:1015A00001231A4362502863054881688022114351
:1015B0008160D3E768030020000002403B7500080B
:1015C000003801400B49C86A401CC8620A480268DA
:1015D0009204D20F05D001225203426000220A6316
:1015E0004A7201688903C90F02D001214904416090
:1015F00070470000FC0300200000024010B50029E5
:1016000010D0C26843685218934200DCD21A0023FB
:101610004361C2608468944204D101228261836084
:10162000C360C361084610BDFF2109220131D20603
:10163000002801D09162704791617047F8B5164655
:101640000F46054602F062F8701EC00A401C81B2C7
:10165000384602F033F80024761C76080EE060006D
:1016600042195278295C120289188AB2C1190023E2
:10167000022001F0EFFF002802D0641CA642EED841
:10168000054A1169802319431161002801D0002007
:10169000F8BD0120F8BD00000020024070B50C46E6
:1016A000054602F033F8A1B2284602F007F80348D5
:1016B0000169802211430161002070BD00200240B9
:1016C0000A07120F01219140014201D00120704709
:1016D000002070470A07120F01219140014201D0FA
:1016E0000120704700207047F8B50B051B0E254CF4
:1016F0005B001C1909239B01E31800930523DB0100
:10170000E618012307469B020A07E5180020120F7E
:101710003B0004F009FE09060A0E12191D21282FAC
:101720002E00FF2928D800981BE0FF2924D8009814
:1017300008E0FF2920D8B08A18E080291CD20F20A9
:1017400080012018808E11E0802915D2A88A0DE032
:10175000402911D2B08E09E040290DD20B20800122
:101760000EE0808A02E0802906D2A88E1146FFF79B
:10177000B1FFF8BD802901D30020F8BD0920C001C8
:101780002018EEE700110020C1688268914201DA5A
:10179000501A7047914202DC4269002A02D0406828
:1017A000401A704780690028FBD000207047C2684B
:1017B0008168914201DA501A7047914202DC8269D5
:1017C000002A02D04068401A704740690028FBD0C8
:1017D0000020704707490122896952030818010156
:1017E000914202D3FF38FF38023803490001401804
:1017F000704700003C01002000D0000800B5082020
:1018000000F0D2FC00BD0000F0B5334C4B001C19B9
:101810000923DB01E5180B230246DB010020E31856
:10182000892A25D00EDC2C4F2C4B4E00F619F618C9
:10183000803A130004F078FD091F1F152125292E79
:10184000333A15008D2A3FD00CDC8A2A33D08B2AFC
:1018500035D08C2A05D140293ADA0B208001201896
:10186000808EF0BD992A03D0A12A01D0FE2AF8D19A
:1018700080292DDA2EE00846F0BD102928DAB08A3A
:10188000F0BD102924DAB08EF0BD102920DA052031
:10189000C00108E008291BDA0F208001DFE70829D2
:1018A00016DA012080022018808AF0BD80290FDA24
:1018B0003420285EF0BD80290ADAA88AF0BD4029CC
:1018C00006DA0D208001CAE7402901DAA88EF0BDB2
:1018D0000020F0BD988EF0BD0011002040020000F5
:1018E00010B5074A106A074B9969146AA04201D0E3
:1018F000106A9969044A51430914401A10BD000046
:101900006C01002000E000E05505000031B500F05A
:101910000BF8009C0546601C00D0641C00F004F825
:10192000401BA042FAD338BD014800687047000050
:101930004402002002480168491C01607047000011
:101940004402002010B506480168102211430160CE
:10195000002000F007F800F017F8002010BD00008C
:101960000020024010B5044600F040F97D21C90076
:10197000FFF7BCFB00F07AFB00222146501E00F06E
:1019800025F8002010BD000008B50F48816901222C
:1019900011438161816911400091C26901040A43C8
:1019A000C261C0690022084000901146501F00F03B
:1019B0000DF800221146901E00F008F80022114692
:1019C000501E00F003F808BD0010024010B502F0F0
:1019D00049FD10BDF8B504460068364DC00354D526
:1019E000E8690026C00007D4E86929040843E861D3
:1019F000E8690840012600902F480168C90511D404
:101A0000014608688A1510430860FFF78DFF0746F6
:101A100004E0FFF789FFC01B642823D8264800682C
:101A2000C005F6D5286A0321090208401FD0626864
:101A30000A4082421BD0286A2A6A8843012109048D
:101A40000A432A622A6A8A432A622862C0070ED0A1
:101A5000FFF76AFF074607E0FFF766FFC11B17485D
:101A6000814201D90320F8BD286A8007F4D5286A8D
:101A7000032109028843616808432862002E04D0CC
:101A8000E869012109078843E8612078C00705D08B
:101A9000286BA168800880000843286320788006AE
:101AA00005D5286B10218843E1680843286300208E
:101AB000F8BD0000001002400070004088130000D4
:101AC000F8B5044644480E460068C007C00FB0424F
:101AD0000AD2414801684908490031430160006861
:101AE000C007C00FB0425CD120783C4F800705D5BD
:101AF0007868F0218843A168084378602078C0079F
:101B00003FD06068012813D03968022813D08907B4
:101B1000002946DA79688908890001437960FFF76E
:101B200003FF0546606801280DD0022817D024E085
:101B300039688903ECE78901EAE7FFF7F5FE411B05
:101B40002748814217D878680007800F0128F4D110
:101B500017E0FFF7E9FE411B214881420BD8786866
:101B60000007800F0228F4D10BE0FFF7DDFE411BD8
:101B70001B48814201D90320F8BD78680007800F17
:101B8000F3D115480168C907C90FB1420BD90168E3
:101B900049084900314301600068C007C00FB042E6
:101BA00001D00120F8BD2078400706D578680721CC
:101BB00009028843E1680843786000F01DF87968FD
:101BC000084A0906090F515CC8400749086000200F
:101BD000FFF7C8FE0020F8BD0020024000100240C0
:101BE00088130000E07A00084002002001480068E5
:101BF000704700004002002030B514A00FC889B023
:101C00006C460FC415A00FC80FC4184D6A680C208D
:101C100011460140164B042910D0164808290ED150
:101C20009102090F6C46645CE96A04AD0907090F6B
:101C3000D203695C920F022A03D003E0184609B070
:101C400030BD1846FFF752FA6043F8E70203040577
:101C5000060708090A0B0C0D0E0F101001020304F1
:101C600005060708090A0B0C0D0E0F1000100240A4
:101C7000001BB70000127A00FEB504460078D54D6F
:101C8000C00748D068680007800F012819D068682D
:101C90000007800F022804D16868C003800F022863
:101CA0000FD0012160680904012811D08A000028A2
:101CB00001D0052816D028688843286028689043FA
:101CC00008E02868800326D56068002873D022E0E9
:101CD0002868084328606068002810D0FFF724FEB9
:101CE000064608E0286810432860F1E7FFF71CFE6D
:101CF000801B642870D828688003F7D50BE0FFF7B5
:101D000013FE064604E0FFF70FFE801B6428F1D89F
:101D100028688003F7D420780126800700283DDA60
:101D200068680007800F13D068680007800F0228DA
:101D300004D16868C003800F012809D0E06800283A
:101D400028681CD030432860FFF7EEFD07460BE003
:101D5000286880070BD5E06801282CD107E0FFF741
:101D6000E3FDC01B0228C5D828688007F7D528687E
:101D7000F82188432169C900084328600EE0400823
:101D800040002860FFF7D0FD074604E0FFF7CCFDD8
:101D9000C01B0228AED828688007F7D42078000737
:101DA00023D5E0690028686A0FD030436862FFF7E6
:101DB000BBFD074605E00AE1FFF7B6FDC01B0228A0
:101DC00098D8686A8007F7D50FE04008400068623D
:101DD000FFF7AAFD074605E0A4E0FFF7A5FDC01B3D
:101DE000022887D8686A8007F7D42078042740073C
:101DF000002860DA00200190E869C00008D4E86992
:101E0000B9060843E861E8690840009001200190A4
:101E100071480168C90511D4016882151143016038
:101E2000FFF782FD009005E0FFF77EFD0099401A64
:101E3000642877D868480068C005F5D5A0680128EF
:101E40000AD0002801D0052810D0286A4008400098
:101E50002862286AB84301E0286A30432862A068F3
:101E6000002812D0FFF760FD00900AE0286A38438E
:101E70002862F1E7FFF758FD0099411A574881425F
:101E800050D8286A8007F5D50DE0FFF74DFD00908A
:101E900006E0FFF749FD0099411A5048814241D8B8
:101EA000286A8007F5D40198002804D0E869012148
:101EB00009078843E8612078C0063CD5606901289D
:101EC0000CD0401D686B23D038436863686B4008B2
:101ED00040006863FFF728FD064629E0686B384339
:101EE0006863686B30436863FFF71EFD064604E0D5
:101EF000FFF71AFD801B022862D8686B8007F7D5B0
:101F0000686BF8218843A169C9000843686312E03F
:101F1000B8436863696BF8208143A069C00001433E
:101F2000696308E04CE0FFF7FFFC801B022847D8FC
:101F3000686B8007F7D4206A002846D069680907D3
:101F4000890F022943D001273F060228286805D0BF
:101F5000B8432860FFF7E8FC044633E0B843286044
:101F6000FFF7E2FC064604E0FFF7DEFC801B0228D8
:101F700026D828688001F7D4E86AE16A00090001E0
:101F80000843E862616AA06A084369687B22D20359
:101F9000914308436860286838432860FFF7C4FC11
:101FA000044604E0FFF7C0FC001B022808D828689C
:101FB0008001F7D509E0FFF7B7FC001B022801D923
:101FC0000320FEBD28688001F5D40020FEBD01205D
:101FD000FEBD0000001002400070004088130000A9
:101FE000042204490428086902D09043086170471C
:101FF0001043FBE700E000E0154801686431016030
:1020000014480168491C016013490868401C0860B5
:102010001249134AC868401CC860904216DB002071
:10202000C8601048816D491C8165016D491C0165BE
:10203000416D491C41650C49088B002806D0401EA3
:1020400080B20883782801D978200883704700007F
:102050008C0100208801002024010020AC01002018
:102060001027000080160020B4180020094910B580
:10207000401E884201D9012010BD074C6061032138
:10208000081F02F0EFF90020A06107202061002066
:1020900010BD0000FFFFFF0000E000E010B5FFF7FB
:1020A000ABFF10BDFEE7000010B500210F4A084647
:1020B000516043009B18401C1981FF28F9DD002066
:1020C00005230B4ADB014400A418E418401CA1823C
:1020D0001028F8DB00200923DB014400A418E418D1
:1020E000401CA186FF28F8DD002010BD780E0020DE
:1020F0000011002010B5402802DB0020C04310BDB5
:1021000010221143C200094B4000D218C0185824B5
:102110000D23A1529B010021C3189986E300C0182A
:102120008186034800685065084610BD00110020F4
:102130004402002070B504461E463830049D04F069
:10214000CFFB20462A463146583004F0C9FB002018
:1021500070BD000070B5104D064601462846FEF7DA
:10216000DBFF0E4CE062FFF741FD2946FEF7BEFFA4
:1021700060620B48314600680546FEF7B7FFA06273
:102180002A46002307480F21FEF7DAFF2080E06A85
:1021900064302062002070BD40420F006C010020BE
:1021A0004002002000004042F8B572B6012212033E
:1021B0000921C9068A6200BF00BF00BF00BF8A6153
:1021C000C117490F0818C01084460020104E03465E
:1021D000009017E008200E4C002280218502103C60
:1021E00037687F0400D50A43A562490800BF00BFD5
:1021F00000BF00BF00BFA561401EF1D1D0436946BA
:10220000C8545B1C6345E5DB62B60098F8BD00006E
:10221000100400480B01194930B55B18FF33097FE2
:1022200011331970022159701449002020310C7F9C
:102230009C704C7FDC708C7F1C71CC7F5C710C4679
:10224000203425789D716578DD710B7F15795B19D8
:102250000B774B7F55795B194B778B7F95795B19A2
:102260008B77CB7F157A5B19CB772178937AC91856
:1022700021706178D27A8918617030BD100A00200F
:10228000034610B50020024602E09C5C6040521CF0
:102290008A42FADB10BD000000B50B0004F044F8E0
:1022A00008111111111111110511074907480A8C64
:1022B0008286828A0A80C28A4A80028B8A80408B08
:1022C000C880002000BD0000280C00204013002022
:1022D000F8B508460D460978552901D0252903D0BF
:1022E000012A01DD451C521E344F602479792B7878
:1022F0006143334C0919334C252B30D0A3685B1C48
:10230000A360CB695B1CCB61B97800290FD0F97849
:1023100000290FD001292C4913D007231B02C9180B
:102320000A7501462948FEF742FF0020F870002098
:10233000C043F8BD2549264B55390A750146224848
:1023400007E037235B01C9180A750146204B1E4878
:102350002033C018FEF72BFFF878401CE6E76E79B3
:10236000802E06DDE068401CE060086A401C0862C0
:10237000DDE7334608339A4208D2086A401C0862F7
:10238000E068401CE0600220C043F8BDB11DFFF7CB
:1023900077FFA919897981420DD02069401C2061FD
:1023A00079796020414306480818416A491C416216
:1023B0000320C043F8BD0020F8BD0000EC00002061
:1023C000900600207C040020001100201518002039
:1023D000D506000010B50020124C03462071D2B281
:1023E000002905D021706370A370A272E37005E02C
:1023F000237001216170A370A272E2700A4C002266
:102400006021514309194B608B600B614B618B61FB
:10241000CB610B628B624B62CB62521C0B63092A4D
:10242000EEDB10BD100A0020900600200C20414376
:1024300007480818002150300180418008220271AD
:102440004271817101728172C17208467047000049
:10245000100A0020F8B50E4604462520069F079D69
:10246000089920706270A670E37027712F460020D3
:1024700008376619372B30D01FDC332B1CD006DC15
:10248000002B19D0312B28D0322B15D125E0342B3D
:1024900012D0352B10D0362B0ED16571002D03D004
:1024A0002A46A01DFEF783FEA91D2046FFF7E8FE81
:1024B000B0710D20F0713846F8BD612B0DD006DCEF
:1024C000382B0AD0412B08D0422BF5D105E0622BE6
:1024D00003D0632B01D0642BEED16571E0E70000DF
:1024E000F1B584B0FFF720FA0546FFF7F9F9664E1B
:1024F00004463079002802D0012802D004E00120EF
:102500003071049800F098F93079022801D1032045
:1025100030715E48C179002906D0017A002903D0C4
:10252000C168611A322905D8C1687D22611AD200BA
:10253000914266D95548007A5549002864D05348DD
:102540006023407901225843524B1A50642048645A
:102550004E4E7079401CC0B27071F17A884208D931
:10256000706A7462201AB062B079401CB0710120A8
:1025700070714948727981184348CB7F8038037065
:1025800020310B7843704B7883708978C170057166
:10259000290A4171290C8171290EC1716B46F460C1
:1025A0001978B37989089B0789009B0F19436B46FB
:1025B00019706023374C5343E358002B61D0EF234D
:1025C00019406B4619700823019300910290412332
:1025D00000213248FFF73EFF02463049049803F0DD
:1025E00057F870796021484300194168491C4160DF
:1025F000C268F1688A1A4263C16000203563F071D5
:102600003072002005B0F0BD204B186A401C1862E3
:1026100023484268521C42605E7960203746464338
:102620001C4830180269521C02614269521C426106
:10263000DB79002B02D1836A5B1C836283699A4237
:1026400000D98261134B032A82D900209851C822F5
:102650008A6411490E46C855183E307D002800D1C5
:1026600076E7002337691A4605210498B847307D7C
:102670000028F5D0002336691A4607210498B04790
:1026800066E7102319439CE7100A0020EC000020A5
:102690008016002090060020280C002090050020C5
:1026A0007C040020F8B5844608780C46552801D0F3
:1026B000252802D0012A00DD4C1C60793B4D00909A
:1026C0006979602041433A482B4609188868401CC4
:1026D0008860DF6ADE68E078A278BE1B9B693528D7
:1026E00021D002DC32281ED10AE038281BD002DCBF
:1026F000362818D115E0412815D0422813D114E00E
:102700006E619E4200DDAE612A48A37983540020A9
:10271000CE624861086BB04200D20E63012028727D
:1027200001E00120E8710020F8BD6E619E4200DDED
:10273000AE61204BA17998180646203EF177E179E9
:102740009954217A4170617A8170A17AC170E17ADD
:102750000171217B4171617B817118461838017DBF
:10276000002905D0002306691A4607216046B047B4
:102770006A79602042430E48002116187161686929
:10278000F062316B814200D2306300980E28C5DBC5
:102790002046E77B1030FEF72EFDE17C0002000AA8
:1027A00009060843B90071188863B7E7EC000020F8
:1027B00090060020280C0020F7B515460C46FFF7C0
:1027C0008FF81A4EF06221780020552903D1012D8F
:1027D00001DD641C6D1E317800290FD00127F771CF
:1027E0002A4621460098FFF773FD002805D137726D
:1027F0002A4621460098FFF755FFFEBD7178002953
:10280000FBD00B4E2A46B06B2146401CB0630098AB
:1028100000F060F80028F0D106482A46406C306588
:102820002146009800F0CEF8FEBD0000EC0000202C
:10283000900600208016002070B506460025FFF7A0
:1028400073F8FFF74DF81D4C0122A179002901D141
:10285000A271A062E17900292DD1A16A7D23411ADC
:10286000DB00994227D90021A171216A032902DAEC
:10287000A271A0621FE003291DDD3046E169FFF768
:10288000D5FDE1690C204843021930465032FFF76C
:10289000C1FCE069401CE061A17A88420BDD0220A6
:1028A00020710748017D002905D0002304691A46DC
:1028B00005213046A047284670BD0000100A0020C0
:1028C000100C0020024801610121017500207047B1
:1028D000100C0020F0B508460D460978552901D0A6
:1028E000252903D0012A01DD451C521E2978002329
:1028F0001A4FDB431A4C252906D0A068401CA06063
:10290000386C401C386409E014496E79896C491CA4
:10291000802E05DDE068401CE060B9641846F0BD1B
:10292000334608339A4206D2B964E068401CE0603E
:102930000220C043F0BDB11DFFF7A2FCA91989799F
:10294000814208D02069401C2061F86C401CF8646A
:102950000320C043F0BD0020F0BD00009006002021
:102960007C040020F8B5FEF7BBFF134B1A691979F8
:1029700000291FD05C7A1149002C05D07D208001F0
:1029800048640020587215E00C4E0D4C851A8036B4
:10299000A54204D97D2292018A64012206E012191F
:1029A000904207D97D2292018A6402228A67C86711
:1029B000186930600020F8BDEC000020801600206F
:1029C000E02E0000F7B5087884B00C46552802D1F7
:1029D000012A00DD4C1C6D480168491C01606379C7
:1029E00060786B4903916B49694F0D798037A84234
:1029F00008D0FF2806D0786C401C78640020C043C3
:102A000007B0F0BDA84201D0FF287DD16148C26A5D
:102A1000026101214172E0785F49372874D00CDCF3
:102A20003328FBD004DC0028F8D03128EDD119E0A0
:102A30003428F3D0352867D125E0584BDD1DFF350C
:102A4000FA352A7D2E6961285ED004DC38285BD0F7
:102A5000412859D120E0622856D0632854D06428F8
:102A600052D17EE0A07908704B4820380078A071E0
:102A7000484802612179A01D019300913223029000
:102A80000022294661E0002021793623009101903F
:102A900002460290012158E0A0790870E079487060
:102AA000207A8870607AC870E17AA07A09024018AA
:102AB0009863002A0DD000231A4606210498B047D7
:102AC000287D002805D000232D691A460721049887
:102AD000A84731482F4920388A7A0378A371437870
:102AE000E37183782372C37863720379A3724379A5
:102AF000E37283792373C07960739000E273C01925
:102B0000038F2374038F00E03DE01B0A6374836B23
:102B1000521C1B0CA374806B000EE074D0B2887240
:102B20000A2801D30020887220796A461070C006F6
:102B300003D57D201A4A800190642079A31D0E22BE
:102B40006D460DC54223097900220398FFF782FCE8
:102B50000246F86B401CF8630399049802F098FD54
:102B600011E0E179A07909024018217A647A090418
:102B70002406091940189863002A04D000231A4635
:102B800006210498B04700203AE700007C040020AA
:102B900010060020EC000020480C0020100A002045
:102BA00080160020034610B50020024602E09C5C1F
:102BB0006040521C8A42FADB10BD30B50D46084613
:102BC00009781446252901D0012030BD062C01D2F8
:102BD000032030BD611EFFF7E5FF29192039C97FA9
:102BE000814201D0042030BD002030BD70B51E46AA
:102BF00004460B465520049D059920706370A27011
:102C0000E6702571EE2E10D02A46601DFEF7CFFA31
:102C1000691D2046FFF7C6FF61194871A81D052EE2
:102C200002DA002E00D1002070BD05212046FFF7FA
:102C3000B9FF60710620F2E7FEB516460F4605465D
:102C4000FFF7BBFF040014D0E0B2694608720090A1
:102C500002A90B4801910278401E0178EE23094831
:102C6000FFF7C4FF02460749284602F011FD20463F
:102C7000FEBD32463946284600F006F8FEBD00008B
:102C800029010020F80C0020F7B588B04A78F848F0
:102C9000039242688260421C15788E782D093607AF
:102CA0002D01360F0B7935431570F24A02920078E8
:102CB000039A84460C46624501D0FF2A2FD1214653
:102CC000E7780931EC4A002605914F2F74D02EDCAD
:102CD000EA480121192F70D016DC072F26D008DC16
:102CE000002F1CD0012F55D0032F58D0052F47D1CE
:102CF00083E0112F71D0162F70D0E149172F08688B
:102D00006DD0182F3CD15CE2312F76D008DC212F1A
:102D100067D0222F70D0232FE3D0242F30D14AE365
:102D2000322F03D0332F68D0342F29D1DAE004209A
:102D3000642F7DD012DC562F7BD008DC502F79D049
:102D4000532F78D0542F77D0552F19D1B6E2572F63
:102D500073D0582F72D0632F12D1C9E2692F2DD0B2
:102D600008DC652F6BD0662F2DD0672F31D0682FF0
:102D700006D1D6E26B2F24D0732F70D0742F6FD072
:102D800002206946087404A90191EE232A460090A6
:102D9000614608E0641D00930194012349E2B949AA
:102DA0001820A6E203990298FFF720FF0246029935
:102DB000089802F06DFCFEE237E220E2B2490C20F6
:102DC00097E2B24995E2B1491039502091E23B4671
:102DD0002FE2E1790020A74A08E0C5E1D3E1E9E16B
:102DE0000BE0EFE023185B7A1354401C8842F9DBB8
:102DF000A04803F0DDF9C2E254E1A2796179120240
:102E00008918E27989B2882B2BD0892B2DD08A2B77
:102E10002FD0832B32D0842B35D0852B38D0862BE6
:102E20003BD0872B3ED08B2B41D08C2B44D007E05E
:102E300062E24CE2F7E101E217E2FCE150E268E213
:102E4000FE2B12D0A92B3CD0B32B3ED0992B3FD0D8
:102E5000A12B42D08748103840180092A5E179E2B2
:102E600090E2490009188A483AE04900091889485F
:102E700036E0490009188648203831E04900091831
:102E8000952080002CE0490009189D20800027E053
:102E900049000918A520800022E049000918FD20FA
:102EA00080001DE0490009187948A03818E0490061
:102EB0000918DD20800013E049000918BD208000BA
:102EC0000EE04900091874480AE04900734807E019
:102ED000734849000818001DBFE749000120C006DB
:102EE0000818BAE7A279617912028918E27989B2E1
:102EF000882B23D0892B25D08A2B27D0832B2AD02F
:102F0000842B2DD0852B30D0862B33D0872B36D0F9
:102F10008B2B39D08C2B3CD0FE2B40D0A92B42D010
:102F2000B32B44D0992B45D0A12B46D05148103813
:102F3000401800220599FEF73AF920E249000918E5
:102F400053483DE049000918524839E04900091842
:102F50004F48203834E049000918952080002FE0C0
:102F6000490009189D2080002AE049000918A52081
:102F7000800025E049000918FD20800020E049007C
:102F800009184348A0381BE049000918DD208000DB
:102F900003E049000918BD2080000818C9E749006E
:102FA00009183C48F9E7490009183B48F5E749008A
:102FB0003A48F2E749003A4802E049000120C006D9
:102FC0000818B7E76279A479240212190924A40128
:102FD00092B2002B14D0012B19D0022B23D0032B3B
:102FE00027D0042B2DD0052B31D0062B2FD0082B2A
:102FF00036D06846067404A821230091019018E198
:1030000013095B001818001930E0012025E01309AE
:103010005B001818001912E013071B0F0A469A40AC
:103020001040F2D119E013095B0018180523DB01E9
:103030001BE013095B0018180F239B01C018808E3A
:10304000EAE713095B00181801239B020DE0D20088
:1030500010184030007E4006C00F6A461074CAE760
:1030600013095B0018180923DB01C018808AD3E715
:1030700028010020F80C0020B418002000110020C6
:10308000780E002088700008ACF7FF1F107C000845
:10309000B4040000B4050000B4060000900600204F
:1030A00080100020A2796179120289188DB2002B5C
:1030B00017D0012B1ED0022B25D0032B2CD0042B94
:1030C00033D04021052B38D0062B36D0072B3FD0EC
:1030D0006846067404A80190B84800960278222336
:1030E00060E62B095B0029071B18090F9520E27980
:1030F000800035E02B095B0029071B18090F9D2074
:10310000E27980002CE02B095B0029071B18090FCE
:10311000A520E279800023E02B095B0029071B181A
:10312000090FFD20E27980001AE029072B09090F19
:103130005B001B18E279A24812E0EA001018403048
:10314000028B8A43E179C907490E0A430283C1E72A
:103150002B095B001B1829079948E279090F803079
:10316000181802F0B9FAB5E7002B02D0012B03D0F2
:1031700005E102F0A7FC02E102F06CFCFFE08F48E1
:10318000E37802780EE6A179607909024018E179C6
:103190008C4C80B2002B0AD08B4E012B02D0928A2D
:1031A000002A04D040008019009101900FE64000F1
:1031B0000019F9E7002800D00E6000961723019649
:1031C00037E0002800D00E60A1796079090240182C
:1031D00085B2E27900207D4903E027187F7A0F54F9
:1031E000401C9042F9DB7949284603F009F809347C
:1031F000724800960196049402781823D2E5A379C8
:1032000060791B02C018D082908A002809D096826B
:103210006F4802F0FDF9694800960196027819237B
:10322000C0E59182F4E7138300E0168300960196CF
:10323000E3782A46B6E5664920205AE0A17960790C
:1032400009024018634980B20A18E179121D7828F2
:1032500001D3002105E00B18782B02D97821081A38
:1032600081B2C8B201920090B1E5A17960790902FA
:103270004018584980B20B18E2791B1D782801D3F9
:10328000002205E01118782902D97821081A82B2A3
:1032900018460599FDF78BFF009601964748E3789D
:1032A000027803990298FFF7A1FC02460299089858
:1032B00002F0EEF9474802F0C3FF7CE0454802F017
:1032C000BFFF3E4800960196027855236AE54048C4
:1032D00002F09EF93948009601960278562361E57E
:1032E000032109023C48FDF77BFF009601966EE53D
:1032F0003A49019100906AE5A17960790902401884
:10330000E17980B20D01FEF765FAE9B20091019012
:1033100035E7FEF7F5F8294800960196027865230F
:1033200040E5009665232A46019603990298FFF727
:103330005DFC02460299089802F0AAF9012080F388
:103340001088BFF34F8F27492548C860BFF34F8FC0
:1033500000BFFDE7A17960790902401880B2E279E7
:10336000059902F033FF002809D0C0B2009004A9EB
:10337000124801910278EE23401E017813E5009671
:103380000196FCE6A17960790902401880B20690A6
:10339000E47900963B462A46019603990298FFF786
:1033A00025FC02460299089802F072F92246059916
:1033B000069802F01BFF00200BB0F0BD2901002091
:1033C000140400000080000800A00008F80C002091
:1033D000B41800208010002090060020F416002071
:1033E0000400FA0500ED00E070B5FEF753F816484A
:1033F00000F0EAFA154D164C6869A065124881681C
:1034000061658188491C81808088E0640E4802F0F3
:10341000FFF82868206768686067A868A0670122CD
:103420000C4B1146A06DFDF7D9FF20468030E968AE
:103430000160A9694160E96981602969C160296AFF
:103440000161002070BD0000B41800203C01002084
:10345000801600203930000030B583680122134007
:1034600002D00022104630BD8C684B68C9682343E7
:10347000C468034D2C4021430B43C360F2E70000B6
:10348000C73FFFFF30B583680122134002D00022FE
:10349000104630BD18C94D6823430C6889682C4319
:1034A00023430B43C168024C21400B43C360EFE749
:1034B0003CC2FEFF08B504494A6902434A614969B2
:1034C0000140009108BD00000010024008B5044909
:1034D000CA690243CA61C9690140009108BD000080
:1034E0000010024008B504498A6902438A6189696B
:1034F0000140009108BD00000010024070B5094E67
:1035000004467618203E049D0C34F17F0830102DBF
:1035100003D00A50F07F035170BD0A51F17F0B5068
:1035200070BD000030710008044A51182039C97F6D
:103530004258520852004250704700003071000853
:10354000044A51182039C97F425801231A43425076
:103550007047000030710008044A51182039C97FB3
:10356000425802231A43425070470000307100084D
:10357000054B10B559182039C97F4358032424033B
:10358000A3431343435010BD36750008054B59182B
:103590002039C97F001D0B581B0C1B0413430B5013
:1035A0007047000030710008054B10B559182039DC
:1035B000C97F4358034C23401343435010BD0000C0
:1035C00036750008EFBFFFFF054B10B559182039BD
:1035D000C97F43588024A3431343435010BD0000C8
:1035E00036750008054B10B559182039C97F435866
:1035F0000324A402A3431343435010BD36750008AF
:10360000054B10B559182039C97F43582024A343CE
:103610001343435010BD000036750008054B10B52C
:1036200059182039C97F43584024A34313434350BA
:1036300010BD000036750008054B10B5591820392B
:10364000C97F435803242402A3431343435010BDAE
:1036500036750008F0B51FB40024022804D00128F4
:1036600004D00425144F12E00125FBE70225F9E7F9
:10367000019861000E18220103990298FDF786FD5A
:1036800039690122114339613080641CE4B2AC42D3
:10369000EED3F868C007C00FFBD1F8688006C00FF2
:1036A00008D0F86820210843F860386940084000D5
:1036B0003861012005B0F0BD00200240C90210B5FC
:1036C0000B1811491AE00C69022214430C6148617D
:1036D0000A69402422430A61CA68D207D20FFBD18B
:1036E000CA689206D20F0DD0CA6820242243CA604D
:1036F0000C69022294430C61920280189842E2D332
:10370000012010BD002010BD002002400748C16804
:10371000C907C90FFBD101698022114203D00449B6
:1037200041600449416001207047000000200240D0
:1037300023016745AB89EFCDF0B500233CE00124C0
:103740009C40224037D04F680668144654436500B9
:103750006519AE4367433E4306604E68012E01D0B3
:10376000022E05D18F6886686743AE433E4386606C
:103770000F69C668AE4325467D432E43C6604D683B
:10378000022D18D14D69FF2A09D8066A54435443C3
:103790002201121B96436C43264306620BE0140A77
:1037A00022466243624362431401A61A446A6A4392
:1037B000B443144344625B1C0A681446DC40BED127
:1037C0004A68012A01D0022A06D10A68C9684368FA
:1037D00093434A43134343600120F0BD10B50446B0
:1037E00001F04AFD206001F02DFD606001F038FD20
:1037F000A06010BD014610B5002000290FD1104A6D
:10380000116B8907890F01290AD0022911D00329D8
:1038100009D001F031FD01F015FD01F021FD10BDD1
:1038200001F02AFD10BD11688907C90FFAD00548BB
:1038300010BD116A8907C90FFAD00120C00310BD5D
:103840000010024000127A00F0B50268194B1A4CC1
:10385000984201D0A04203D17025AA434D682A4363
:10386000164D174E174F98420AD0A04208D0164C5A
:10387000A04205D0A84203D0B04201D0B84204D142
:1038800003242402A243CC68224302608A68C262F5
:103890000A888262984205D0A84203D0B04201D083
:1038A000B84201D1097C01634169012211434161A0
:1038B0001046F0BD002C01400004004000400140D3
:1038C00000440140004801400020004041680122BE
:1038D000D202914341608168082291438160704720
:1038E000FEB5044600680D460026C007C00F4FD144
:1038F000E9686868AA69084329691143084321688F
:10390000244A114008432060A8686168032212031A
:103910009143014361606869A168121191430143B9
:10392000A1601D48844203D10020FFF763FF12E02D
:103930001A4884420BD01A48844208D0194884425D
:1039400005D01948844202D01848844220D16846E4
:10395000FFF744FF029800281AD02968002917D0E1
:103960000126AA69F3039A420CD140004A08801844
:10397000FDF7BCFB0E4980B201400007420F0A432D
:10398000E26005E04A081018FDF7B0FB80B2E06085
:103990003046FEBDF369FFEF0038014000440040AF
:1039A00000480040004C004000500040001401401E
:1039B000F0FF000010B580220249FDF7F8FB00205F
:1039C00010BD0000A0700008F0B5154A00211514C4
:1039D000144C154F0CE0D65ABE4208D19B185B8898
:1039E0006668B34203D90AC44B1C2360083C491CD7
:1039F0004B01AB42EFD321680123002905DB4901CC
:103A00008918202201F0D2FC00E08380A0684001E8
:103A10002030A84201D90020A0600020F0BD0000A5
:103A200000C800083C010020AA5500001FB50B4645
:103A3000024604A1684602F063FC0146684601F0B4
:103A4000DFFB1FBD201B5B25643B25644800000095
:103A500070B501208AB04002FFF744FD224CA06AF5
:103A600003263043A0622149B0050A68824302431D
:103A70000A60A26A83111A43A2620A68824302435F
:103A80000A60002505950695079505A92046089525
:103A9000FFF7E2FC0120039000950195029569462D
:103AA00004952046FFF7EEFCE16804208143E160C5
:103AB0006169C908C900314361616168014361609E
:103AC0006068082188436060A06817218843C9079F
:103AD0000843A060A068C00FFCD1A068044908405A
:103AE000401CA0600AB070BD0024014008270140BE
:103AF000E8FFFF7F10B50120FFF7DCFC00210A2062
:103B000000F08EFC0A2000F081FC00210B2000F068
:103B100087FC0B2000F07AFC10BD0000F0B50120FE
:103B200087B04004FFF7C6FC01208004FFF7C2FC09
:103B30000120C004FFF7BEFC01208005FFF7BAFC9E
:103B40001C480125002403266A46049551C2092712
:103B5000FF0669463846FFF7EFFD1920000203947F
:103B60006A46049461C269463846FFF7E5FD2802BB
:103B7000B86111486A46049551C2104F69463846EB
:103B8000FFF7DAFD0B20000303946A46049461C238
:103B900069463846FFF7D0FD0720400300900294A5
:103BA00003946946019504940548FFF7C5FD07B0E5
:103BB000F0BD0000C0800000E743000000040048A2
:103BC00000080048084807490160084901600421CD
:103BD0004160074A8260C1684907FCD1026105491A
:103BE00001607047CCCC000000300040555500000B
:103BF000FF0F0000AAAA000010B586B01421684685
:103C0000FDF7EEFA1020FFF761FC0021112000F013
:103C100007FC112000F0FAFB2F20694608800020E5
:103C200001900848084C02902046FFF70DFE2068DE
:103C3000802188432060E06801210843E06006B0ED
:103C400010BD0000E70300000010004070B5012027
:103C50008EB08003FFF746FC03204002079002204D
:103C60000890032000240990012509200A9407A93F
:103C70000C950B94C006FFF75FFD3A4E102202210F
:103C80003046FFF791FC002202213046FFF770FC1E
:103C9000002202213046FFF7B3FC00220221304609
:103CA000FFF7BCFC802202213046FFF78DFC00228A
:103CB00002213046FFF7C0FC002202213046FFF708
:103CC00091FC002203213046FFF76EFC0022032105
:103CD0003046FFF74DFC002203213046FFF790FCF1
:103CE000002203213046FFF799FC80220321304651
:103CF000FFF76AFC002203213046FFF79DFC0022FB
:103D000003213046FFF76EFC00211B2000F088FBEA
:103D10001B2000F07BFB144869460068009001946A
:103D200002940394059406940C20104C04902046B1
:103D3000FFF7D6FD606829050843606060684900A8
:103D400003225205904308436060A068491208436B
:103D5000A0602046FFF7BAFD2068284320600EB01F
:103D600070BD000000000240DC000020003801406F
:103D7000F0B58DB01C2106A8FDF732FA182168466F
:103D8000FDF72EFA012464042046FFF79FFB20462E
:103D9000FFF790FB012500240E2002260327039540
:103DA0006A4605950494C1C209206946C006FFF71A
:103DB000C3FC00960920039504956946C006029746
:103DC00001960595FFF7B8FC464E102204213046B7
:103DD000FFF7EAFB002204213046FFF7C9FB00226F
:103DE00004213046FFF70CFC002204213046FFF787
:103DF00015FC802204213046FFF7E6FB0022042157
:103E00003046FFF719FC002204213046FFF7EAFB99
:103E1000002205213046FFF7C7FB0022052130466E
:103E2000FFF7A6FB002205213046FFF7E9FB002241
:103E300005213046FFF7F2FB802205213046FFF7CF
:103E4000C3FB002205213046FFF7F6FB00220521C7
:103E50003046FFF7C7FB00211C2000F0E1FA1C20D0
:103E600000F0D4FAA61EFF21304600F0D9FA304601
:103E700000F0CCFA1C48EE03006806900794089402
:103E800009940C200AAA51C2184C06A92046FFF733
:103E900027FDA06821140843A060A068B043304308
:103EA000A06020681F2149058843084320602068DE
:103EB0004911884308432060606829050843606011
:103EC000606849007A05904308436060A068491221
:103ED0000843A0602046FFF7F9FC206828432060D3
:103EE0000DB0F0BD00000240E000002000440040A2
:103EF00030B58DB01C216846FDF772F9182107A86E
:103F0000FDF76EF90124A4042046FFF7DFFA2046EE
:103F1000FFF7D0FA032080020790022008900320C8
:103F20000024012509A931C104200C9007A91348D8
:103F3000FFF702FC00211D2000F072FA1D2000F0A6
:103F400065FAE120800200900C2001940294039411
:103F500005940490E8030A4C069069462046FFF752
:103F6000BFFCA068A1140843A0602046FFF7AEFC88
:103F70002068284320600DB030BD000000040048D8
:103F80000048004010B58EB01C216846FDF728F9A6
:103F9000182107A8FDF724F901200005FFF796FA7C
:103FA00001208004FFF786FA18200790022008906D
:103FB00003200990002404200C900A940B9407A974
:103FC0001348FFF7B9FB00211D2000F029FA1D203E
:103FD00000F01CFAE120800200900C200490019473
:103FE0000294039405940120C0030A4C069069468C
:103FF0002046FFF775FCA068A1140843A060204686
:10400000FFF764FC20680121084320600EB010BD5A
:10401000000400480050004030B58DB01C216846B7
:10402000FDF7DEF8182107A8FDF7DAF82020FFF7E2
:1040300059FA01204004FFF73DFA30200790022092
:10404000089003200990052000240C9009200A9470
:104050000B9407A9C006FFF76FFB00211D2000F09D
:10406000DFF91D2000F0D2F9E120000200900125C7
:104070000194029403940C20ED0304AA31C20B4C6A
:1040800069462046FFF72CFC6068A843284360601F
:10409000A068A1140843A0602046FFF717FC206821
:1040A0000121084320600DB030BD00000014014024
:1040B00000B50846042A02D80020C04300BD01789C
:1040C0007F2902D90120C04300BD41784906490E2D
:1040D0001F2902D90220C04300BD114602F0CAFBCD
:1040E0000028F9D0042000BDF7B588B00F460A9A21
:1040F0000898FFF7DDFF0690002803D00020C0439A
:104100000BB0F0BDBD483A7800783946824273D191
:104110008C784A78CB78B98824024DBAB8491C43C8
:1041200008704A7001200790200521070226000E22
:10413000090F130002F0F8F811A60A508DA7BFDD91
:10414000A6A6A6A6A6A6A6A6E9F0A600E81DC008F3
:10415000AB4903908870002038E0002701200597C4
:1041600001900098C000049026E021070122200958
:10417000090FD202944207D24200A2481218092025
:1041800080011018808E05E042009E481018FF3014
:104190008130808AFDF794FA002801D00198074306
:1041A0000198641C4006000E01900598A4B2401CC2
:1041B0000590082804DA049805994018A842D4DB31
:1041C0008F4800994018C7700098401C03990090D0
:1041D0008842C2DB761854E0E81DC0088849039085
:1041E0008870002030E000200090012001900298AB
:1041F0000027C00004901DE0FDE02005000E4200F5
:10420000804821071218092080011018090F808AA0
:10421000FDF756FA002803D0019900980843009052
:104220000198641C4006000E7F1CA4B20190082F68
:1042300003DA0498C019A842DFDB7149029A00989A
:104240008918C8700298401C039902908842CADB02
:10425000C0E768006A498446887000200EE0211893
:104260004A006849470052180921C9015118898E2E
:10427000634A0B0ABA18D3701171401CA842EEDBD6
:1042800017E0761C8DE068005D4A8446907000203F
:104290000DE021184B005B4947005B18092189019B
:1042A0005918898ABF180B0AFB703971401CA84243
:1042B000EFDB6644E5E7002D12D0FF2212029542A3
:1042C00007D142004F4812189D208000101801F0BD
:1042D000FBF939464A480A9AFCF769FF0A9E85E0CD
:1042E0004200484812189D208000101801F0ACF8D8
:1042F000EFE73879797900020843424962005218A1
:104300000921C90151188886E3E7E81DC0083C4926
:1043100003908870002036E047E03818C07900909C
:1043200001200190002005900298C000049024E034
:10433000210701222009090FD2029442009B019A11
:1043400007D21A4043002F481B189D2080001818E0
:1043500005E01A4043002B481818FF30953001F053
:10436000C7F90198641C4006000E01900598A4B29C
:10437000401C0590082804DA049805994018A842C2
:10438000D6DB0298401C039902908842C5DB1C488A
:10439000B9788170F978C170397901717979417191
:1043A000361D0698002814D025E000200EE04100BC
:1043B000C919CA79097A12020A4321184B00114916
:1043C0005B180921C90159188A86401CA842EEDBF6
:1043D000DDE70798002809D0B1B2094802F04AFA8F
:1043E00007498855000A89194870B61C32460449A5
:1043F000089801F04DF9002082E600003401002009
:10440000F80D00200011002070470000C106C90E01
:1044100001208840014908607047000000E100E089
:104420008307FF22DB0E9A408907090E9940002876
:104430000BDA0007000F0838830808489B0018189B
:10444000C36993430B43C3617047830804489B00CF
:104450001818036893430B430360704700ED00E0B6
:1044600000E400E08307FF22DB0E9A408907090E73
:10447000994000280BDA0007000F08388308084825
:104480009B001818C36993430B43C36170478308AB
:1044900004489B001818036893430B43036070475C
:1044A00000ED00E000E400E0F7B58CB000200B90D8
:1044B0000D98007854280ED10D984078C006C00E93
:1044C0004100411805900020C0430B31914203D1B7
:1044D0000598022802DA00200FB0F0BD0D9841794E
:1044E00002790802104380016421FCF7FFFD069069
:1044F0000D982230417A027A08021043800164212B
:10450000FCF7F4FD0699814204DBCD48816B491C20
:104510008163E0E7401A0599491EFCF7FDFD0A900A
:104520000C98002863D1C6488168491C002481602A
:1045300058E0600021180D98069A08180A996143FE
:104540008D18BF490A69521C0A613721C9018D4281
:1045500002DABB4B01221A706A1A232109028A422D
:104560002CD2017A1E293CD3C17980790E020643F0
:10457000284602F025FD7D27FF0070433946FCF7F1
:10458000CBFD0090284602F037F971424843394686
:10459000FCF7C2FD0146AA483746006A0C220346D2
:1045A000A84E53439A199760009FF7505160FF211E
:1045B0009031884202DAA249401C08627D20C00185
:1045C00085420EDD9E4D2878012807D12A6A002AEF
:1045D00004DD9C490020AA6100F076FC00202870D0
:1045E0002862641C0598844201DA282CA1DB0C980F
:1045F00001287DD19248C168491C0024C1600BE1AB
:104600000A9A069B62436000D51821188C4B0D98BE
:104610005A690818521C3726017AF6015A61B542C8
:1046200002DA874A012353702322AB1B1202934202
:104630002DD21E297ED3C17980790E0206432D200A
:104640000002281A009002F0BBFC7D217043C900D3
:10465000FCF762FD0746009802F0CEF87D2170431A
:10466000C900FCF759FD024675480C23416A08460B
:104670005843754B8446C018866066469F51426019
:10468000FF209030814202DA6D48491C41627D2052
:10469000C00185424EDD6A48407801287ED1684DD0
:1046A000686A0990002879DDE86168480390002075
:1046B00008907D20C000424200238446049201926B
:1046C000009063491A46184607931BE00C255E4E7E
:1046D0004543AF19BE680296322E12D37F685A4EF8
:1046E000282F0EDB75595B4EC835B54209D200E064
:1046F00098E08F4200DA3946039E029DB54200D20F
:104700000395401C099DA842E0DB00254EE00C20EB
:104710002E464D4F4643B859F71903907E680296CE
:10472000BE68322E41DB029E282E3EDB0646C8368E
:10473000484F00E06FE0BE4237D20E46029F32364D
:10474000B7420BDD002B01DD002A03D0002A2CDD4F
:10475000002B2AD10798401C079026E0089E3D4F69
:10476000761C08960646C736BF1EBE4207D2009F7B
:10477000B84200DA0090019FB84200DD0190FF27A7
:104780002C37BE4205D2049F039EBE4200DD04903A
:104790005B1C0646C93EFF272C3700E037E0BE42CF
:1047A00003D2604500DA8446521C6D1C099885428C
:1047B00003DAFF20F5308142A9DB0020002B07DD62
:1047C000002A05DD079A002A02DD6046049A04E00B
:1047D000089A0A2A05DD019A00988018C20F10185D
:1047E0004010174B9A6A550052191018C217920FB1
:1047F0001018801098621648814208DA586B4200FF
:1048000080184018C117890F0818801058630C4988
:10481000002048704862641C0598844202DA282C03
:1048200000DAEDE606494A6B086B8018CA6A520046
:104830008018C217920F10188010C8620B984BE6B0
:10484000FC01002034200020F432002003D90000B5
:104850000F270000BD02000010B5040001D0601C4D
:1048600003D10221064801F045FC012C01D0641C53
:1048700003D10221024801F061FC002010BD0000BC
:10488000FE01002070B572B60125094A2D0395611D
:1048900080210C028B019362084201D0946100E0F8
:1048A000946249089361F6D19562956162B670BDD4
:1048B0000004004810B501200449C00648600448BF
:1048C0000168491C016000F005F810BD00ED00E032
:1048D000D800002070B5094DE86F00280CD0084CB6
:1048E000084902202268FDF767FF00202060E86782
:1048F0008021044801F068FB70BD0000FC0300202B
:10490000E80000201005002010B50648054B00788F
:104910000021403B5A1840325478491C14700F292A
:10492000F8DB10BD4011002010B5084C084B0122E7
:104930000221A06DFCF752FD064800F069FEE06D13
:10494000401CE065A06D2066002010BD8016002090
:1049500039300000B41800200248C16D491CC165FF
:104960000020704780160020F3B5FA4D85B0286806
:1049700000286FD0686800281CD000220D21082074
:1049800000F0CCFE00221146082000F0C7FE0122F4
:104990001146082000F0C2FE00200146EE4A13181E
:1049A0004033401C19701028F8DB00260121144602
:1049B00040347BE20122E1E7B2000598059B805C70
:1049C000D7187A78019201257B8800931B2873D031
:1049D00012DC0246030001F0A7FC1B5C72727272CB
:1049E00072723E3E3E3E3E3E5C5C5CA7A7A73E3EEA
:1049F000BEBEBEBEBEBE5C00342870D011DC014617
:104A00001C390B0001F090FC18A7A7A7A7A7A7A720
:104A1000A7A7A7A7454545454545454545454545BE
:104A2000F7453A2873D008DC014635390B0001F010
:104A30007BFC05E26E56E26E3000DC2804D004DC1C
:104A40003B28EFD0C82824D120E1DD28FCD0FA286B
:104A5000F9D11BE133E2D01F030001F065FC0E0821
:104A60000A10181B1D1A1A1A1A1A1A20261A207C44
:104A70004AE0FFF749FF00281FD0207C3AE0FFF70B
:104A800043FF002816D1207C002813D125E000F038
:104A9000A1FBF5E12078F7E7FFF736FF1DE0207C6A
:104AA00000280AD0002905D007E0207C002804D186
:104AB000002902D0012010E04DE000200DE013009D
:104AC00001F032FC070C050E111B262E0C0000F025
:104AD00081FB00990198FCF707FE2074D0E11AE1F0
:104AE00000F078FB0CE0207C0028E6D000990198CB
:104AF000FCF7FAFD0028E0D0DCE7207C0028DCD0C1
:104B000000990198FCF7F0FD0028D6D1D2E758E1D2
:104B1000207C0028CED100990198FCF7E5FDB3E791
:104B2000207C0028ECD0C5E7102804D0112804D040
:104B3000122AAED10AE0227C03E0207C0028A8D013
:104B400001220099019800F0E9FD99E1207C0028FC
:104B50009FD00022F5E715383D79030001F0E4FB12
:104B6000120A1215181B0F1E3C4C5B6A2D798185A9
:104B7000898D7D9400F02EFB13E0207484E000F01A
:104B800029FB1DE000F026FB29E000F023FB36E0C6
:104B900000F020FB42E000F01DFB4EE0207C0028EE
:104BA00070D028460099FCF72FFE0546F9887879E1
:104BB000FCF72AFE854263D064E0207C002861D0A7
:104BC00028460099FCF720FE0546F9887879FCF71D
:104BD0001BFE854254D155E0207C002852D0284647
:104BE0000099FCF711FE0546F9887879FCF70CFE70
:104BF000854245DB46E0B1E0207C002842D02846D3
:104C00000099FCF701FE0546F9887879FCF7FCFD70
:104C1000854235DC36E0207C002833D028460099D8
:104C2000FCF7F2FD0546F9887879FCF7EDFD854241
:104C300026DD27E0207C002824D028460099FCF7B8
:104C4000E3FD0546F9887879FCF7DEFD854217DA41
:104C500018E0207C002813D1A3E7207C00280FD186
:104C6000AEE7207C00280BD1B9E7207C002807D1D3
:104C7000C5E7207C002803D1D0E7207C0028DCD0C9
:104C800001207AE7002078E70225F9E03F79154610
:104C9000C8280DD0DC2823D0DD282AD0FA28F3D16B
:104CA0002D48E90008184030007EC0062AD508E0EB
:104CB0002948E90008184030007EC00601D40021D0
:104CC00021E0207C002822D038460099FCF79CFD8A
:104CD0000146284600F0C0FB284600F0D3F94CE717
:104CE0001D48E90008184030007EC006E9D40121C3
:104CF00009E01948E90008184030007EC006E0D4F9
:104D0000022100E003212846FDF7F4F9D9E72846FF
:104D100000F0F8FEE0E73F790225342802D037287A
:104D200016D108E0207C002812D038460099FCF704
:104D30006BFD401C07E0207C002809D03846009914
:104D4000FCF762FD401E02463846009900F05CFD0B
:104D500096E00000780E0020001100203D7979795E
:104D60000291F9880191332814D035281BD03828B6
:104D70008AD1207C002887D00298FCF745FD0746A1
:104D800028460099FCF740FD3A1A0199029800F074
:104D90003BFD79E7207C0028FBD028460099FCF7F2
:104DA00033FD0246F1E7207C0028F2D02846009926
:104DB000FCF72AFD054601990298FCF725FD2A1803
:104DC000E3E73A7979790291F9880191797A039147
:104DD0007D89362806D0392812D03A281FD03B28A2
:104DE0004DD131E0207C002849D010460099FCF7D5
:104DF0000BFD074601990298FCF706FD3A180CE0F6
:104E0000207C00283BD010460099FCF7FDFC0746AB
:104E100001990298FCF7F8FC3A1A29462CE0207C0C
:104E200000282CD010460099FCF7EEFC07B201993F
:104E30000298FCF7E9FC00B247433A46294603983A
:104E400000F0E2FC3A1416E0207C002817D010464F
:104E50000099FCF7D9FC07B201990298FCF7D4FC41
:104E600001B23846FCF758F902B20F4629460398BA
:104E700000F0CAFC3A46691C039800F0C5FC032503
:104E8000301141000F48012308183107090F02892A
:104E90008B401946114000D00121277C0830002F9B
:104EA00001D01A4300E09A430280761906988642A0
:104EB00000DA81E503494868401C4860002007B0DB
:104EC000F0BD0000780E0020F7B586B005927D2277
:104ED00065480024D2008646504200900490039218
:104EE00001926348029404606049234622462046AA
:104EF00019E00C254543079E2F46AD19AE68B44610
:104F0000322E0FD36D68282D0CDB3E46079FBE590D
:104F1000584FC836BE4205D28D4200DA2946F445C4
:104F200000D2E646401C059DA842E2DB681E57E021
:104F300070460C25079E45437059AD196E68AD68E3
:104F4000B446322D4ADB6646282E47DB0646494FDB
:104F5000C836BE4242D20E463236B4450BDB002B79
:104F600001DD002A03D0002A38DD002B36D102985B
:104F7000401C029032E0282C07DA3F4EA700BF19F0
:104F800007263602BE19B580F0803A4E0546C73571
:104F9000B61E641CB54207D2039EB04200DA0390ED
:104FA000049EB04200DD0490FF272C37BD4208D29A
:104FB0000D462835AC4504DA009DA84200DD00907E
:104FC0005B1C0546C93DBD4208D20E462836B44595
:104FD00004DA019DA84200DA0190521C7046401E7E
:104FE0008646002803DBFF20F5308142A0DB204805
:104FF00004604360029D8560C260039D0561009D61
:105000004561019D8561049DC5610020002B08DD7F
:10501000002A06DD029A002A03DD019A0098101882
:1050200004E00A2C05DD049A03988018C20F1018BA
:105030004010124B1A68540012191018C217920F20
:105040001018801018600948401E814209DA0C4A85
:1050500010684300C0184018C117890F0818801045
:105060001060002009B0F0BD03D900001027000037
:10507000B41F0020BD0200000011002038020020F3
:105080002C020020FEB50746402802DB0020C0436A
:10509000FEBD2C48F9000E1800964036348BE10610
:1050A00001D40020FEBDA1063CD561063FD42649AF
:1050B000096800980A25406D0190081AA1070FD0D1
:1050C000A107890F012905D0022905D0E1438907ED
:1050D00005D005E0642503E07D25ED0000E01B4DD3
:1050E000A84224DB2946FCF717F8014615487A0048
:1050F00012180B20800110188446808E019B4018E6
:1051000069435B18009980B24B650D2189015118E4
:10511000898E814203D8084640210C43348361467E
:10512000888604E0600602D5402084433483307EC4
:10513000B9B24006C20F052000F0F0FA307E4006FA
:10514000C00FFEBD00110020440200201027000007
:10515000F7B50446FCF72BFB054602992068A942E7
:10516000A16806DC4018029A0199FCF720F8029920
:1051700019E040182A460199FCF719F829462046FB
:10518000FCF772F92046FCF712FB06460298471B13
:10519000B7420DDCA16820683A46401801994919C8
:1051A000FCF705F839462046FCF75EF90298FEBD8B
:1051B000002E0CDDA168206832464018019949197B
:1051C000FBF7F5FF31462046FCF74EF9AD192846AE
:1051D000FEBD0000074A0F2011183F235B5C4031E1
:1051E000401E0B700028F7DC02494031087C087033
:1051F000704700000011002000B5FFF743FB00BD21
:1052000010B50C460A4601460348FFF7A1FF00F01F
:10521000C3FE204610BD0000C003002010B50C46A0
:105220000A4601460348FFF793FF00F0B5FE20460B
:1052300010BD0000C003002010B50C4600F014FFA4
:10524000204610BD04494968F0221140034A09096B
:10525000515CC8407047000000100240E07A00082E
:1052600003494968034A4905490F515CC8407047E2
:1052700000100240F07A000810B5074841680C2081
:105280000140064805D0042904D0082901D100F0C6
:1052900009F810BD024810BD0010024000127A004B
:1052A000001BB70010B50D4C60680321C903012233
:1052B0000840D203811A0A4802D0914200D109481D
:1052C000E16A0907090F491CFBF710FF61680F220B
:1052D00092041140890C891C484310BD0010024003
:1052E00000127A00001BB7000920C00600694106C1
:1052F000C90FC943C907CA0D012149028A430106E2
:10530000C90FC943C907890D0A430121C00B89028E
:10531000C043C0078A43400D02432248016901206F
:10532000C00282438807C00FC043C007000D02437C
:105330000120000382434807C00FC043C007C00CD0
:10534000024350088A06D30F012240009A431043BB
:10535000022290434A06D20FD243D207920F104343
:10536000042290430A06D20FD243D207520F1043B1
:1053700008229043CA05D20FD243D207120F8905E3
:10538000C90F1043C9431022C9079043C90E0843EF
:10539000054909695202C90BC943C9079043890CE1
:1053A00008437047000400480008004870B5D4174F
:1053B000A40F0023A418A51003E09C000E59065169
:1053C0005B1C9D42F9DCD40F6B00A418651003E050
:1053D0005C000E5B06535B1C9D42F9DC104670BD01
:1053E00000B5FFF781FF00BDF8B500238446802596
:1053F000DB431248002421462A464A4312181788E4
:105400000F4EB74209D17E26B75A0E4EB74204D18D
:105410005288A24201DD0B461446491C0829EBDBE9
:10542000082B06D26B43191880226046FFF7BEFF97
:1054300002E06046FEF7BEFA0020F8BD00C000089A
:10544000AA550000A55A00000B0702881B0F012176
:1054500099408A430280704730B5402802DB002023
:10546000C04330BD0D4CC20013191A464032157EA0
:10547000AD0611D4400000190D24A4010419A18621
:105480000B240021A4010019818605480068586595
:10549000108B202108431083002030BD0011002014
:1054A00044020020034610B50020024604E09C5C44
:1054B0002018521CC0B2D2B28A42F8D310BD0000EC
:1054C00010B50B4C20461E388278611F4A70492265
:1054D000227000796070085CA07003212046FFF7FD
:1054E000E1FFE0700421204600F040F810BD00000C
:1054F000F201002010B51C4C2078002824D0207B1D
:1055000080062DD1607901220023002806D0A271E7
:10551000E07900280AD0401EE07107E0A068401C36
:10552000A0600A2802D91420E071A37160780028D5
:1055300016D02179491CC9B22171814200D922714A
:105540006371FFF7BDFF0BE02069401C2061C82894
:1055500001D9642003E0E079002801D0401EE07109
:10556000E068401CE06010BDD401002010B500F0E0
:1055700009FE10BD70B5044604291AD10321FFF7B6
:1055800091FFE178884214D1184900220878002858
:1055900020780FD00B461433692808D16578087934
:1055A000854204D101254D718A60A2781A54587839
:1055B000C87070BD4928FCD10C4D60784B781E3501
:1055C0009842F6D1A078C87069200A61287048789E
:1055D00068708878A87003212846FFF763FFE87099
:1055E00004212846FFF7C2FF70BD0000D40100204F
:1055F00010B500F001F810BD03488168C907C90F54
:1056000000D0C068704700000030014070470000C3
:1056100070B51A4C6168491C616019490180A18804
:1056200041801849CA6C8280496D81601121818353
:105630001549C183A1684A011449511800250B4638
:105640002A469E5CFF2E04D1521C202AF9D3002D3D
:1056500010D02022FBF7F2FFA0682060401CA06061
:1056600040010121C9022030884201D90020A060F8
:10567000002070BD202200F019FEEDE73C01002063
:10568000AA55000080160020A55A000000C8000896
:1056900010B514460A46012802D0022806D00DE0B3
:1056A00021461046FFF7BAFD054804E021461046A2
:1056B000FFF7C2FD0348816F491C8167204610BD7A
:1056C00068030020FC0300200B0702881B0F012148
:1056D00099400A43028070470907090F01238B4054
:1056E0000188002A01D0194300E0994301807047E6
:1056F00010B5002A02D0FFF7E7FF10BDFFF7A4FEA8
:1057000010BD0907090F01238B400188002A01D031
:10571000194300E0994301807047000070B50B0504
:105720001B0E204C5B000D071C192D0F030000F011
:10573000FBFD09060B14191E22272C313600FF2908
:105740002DD89520800003E0FF2928D89D208000D7
:1057500020182946FFF7D5FF21E0FF291FD8A520F3
:105760008000F5E780291AD2FD208000F0E780292B
:1057700015D20D48ECE7402911D2AD208000E7E7B3
:1057800040290CD2B5208000E2E7802907D20648E4
:105790002030DDE7802902D203488030D8E700209E
:1057A00070BD000000110020140400000121C90395
:1057B000034A002801D09162704791617047000050
:1057C0000008004801218903034A002801D09162A2
:1057D00070479161704700000008004801210922CC
:1057E000C902D206002801D09161704791627047CA
:1057F00001214903034A002801D091627047916159
:105800007047000000080048F0B5304C4B001C19F0
:105810000923DB01E6180B23DB01E51892B28A2885
:105820003DD00EDC294F4B00DF1909239B01FF18E7
:105830008338030000F078FD0714181C21262D463C
:10584000480099283ED006DC8B282CD08C2831D0FB
:105850008D2839D133E0A12834D0FE2834D131E06D
:10586000102931DABA822FE010292DDABA862BE01E
:10587000102929DA0520C00108E0082924DA0F20C0
:10588000800114E008291FDA01208002201882829A
:105890001AE0802918DAB28616E0AA8614E0802978
:1058A00012DAB28210E040290EDA0D2080012018B1
:1058B000828609E0402907DA0B208001F7E74029BA
:1058C00002DAE8E78029E8DB0020F0BD00110020C3
:1058D000F0B58DB0002500F083FFFCF701F80590CE
:1058E00010213A4800F0E6FF0790FBF7F9FF04901B
:1058F0001021364800F088FF0690FBF7F1FF039077
:105900001021324800F09EFF0190FBF7E9FF0646A8
:1059100010212E4800F0AEFF0090FBF7E1FF2C4A6B
:1059200004469068012108439060881E1061294850
:105930001061264B0021585C1070491C1029FADBBD
:105940001768FBF7CDFF0B90019900980297019023
:10595000214F0091781921A1069B079A00F0D0FCF5
:1059600045190B98A11B001B01910290039A049901
:105970000398B21A431A009208460599421A7819F8
:1059800020A100F0BDFC441908A8FDF727FF264818
:1059900042680320C00302403819134623A100F0D7
:1059A000AFFC0419381926A1089A00F0A9FC0119C6
:1059B0003846FFF725FC01210D20FEF737F8244972
:1059C0000320886000200DB0F0BD00005870000872
:1059D0000030024001A00000680200200D0A43527E
:1059E00043202025303458202025303458202025CD
:1059F0003034582020253034582020253034580D9C
:105A00000A00000074696D6520253034642020256B
:105A10003034642020253034642020253034642044
:105A200020253034640D0A00001002404D61696E7B
:105A3000536F75726365202578202564200D0A0058
:105A4000737973636C6B202564200D0A00000000DD
:105A5000C000002030B50021174D084669604200A3
:105A60005219401C1181FF28F9DD00200522134C3A
:105A7000D20143001B199B18401C99821028F8DBA7
:105A800000200922D20143001B199B18401C998653
:105A9000FF28F8DD00201022C100091940310B8BCE
:105AA000401C93430B834028F6DB01200449286007
:105AB0004882002030BD0000780E00200011002038
:105AC000B418002010B500210C48092201600C4BCD
:105AD000084692014400E418A418401CA18610282E
:105AE000F8DB0020012292024400E418A418401CB4
:105AF000A1820828F8DB002010BD0000780E0020ED
:105B00000011002010B5402802DB0020C04310BD6A
:105B10000B4BC100CA18114640310C7EA4060DD5AE
:105B20004000C0180B2300249B01C0188486054840
:105B300000685065088B202290430883002010BD28
:105B4000001100204402002010B5FBF7F3FEFCF723
:105B5000A5FA10BD70B594B030216846FBF740FB44
:105B60000024022501260E94E803099000960520E2
:105B70000F94C0040D9401960A900C9408950B950F
:105B80006846FCF779F8002803D0862115A000F0BC
:105B9000B5FB07200C900E9401210D950F940CA8D5
:105BA000FBF78EFF002803D092210EA000F0A6FB89
:105BB000109610A81296FBF70DFF002803D0A12124
:105BC00008A000F09BFB4B208001FCF74FFA04205B
:105BD000FCF706FA00221146501EFBF7F7FE14B040
:105BE00070BD00002E2E5C5372635C4253502E63D6
:105BF0000000000013480168012211430160416860
:105C0000114A114041600168104A11400160016869
:105C1000012292049143016041683F2212049143A2
:105C20004160C16A09090901C162016BFF22143296
:105C300091430163416B4908490041630021816040
:105C400070470000001002400CB8FF08FFFFF6FE8E
:105C500004480169C907C90F02D00121C943016184
:105C6000704700000010004070B51A4CE0691A4BF4
:105C70008006C00F0BD0A18C5868401C5860184A91
:105C8000164D106829549F2801DA401C1060E06905
:105C90000007C00F09D008202062A0680121090375
:105CA0000843A060D869401CD8612068C006C00FB6
:105CB00007D0E069C006C00F03D01020206200F0BA
:105CC00023F9E0694006C00F03D04020206200F0B5
:105CD0005BF970BD0038014068030020900400208B
:105CE000E400002010B5124CE069E0690007C00F25
:105CF00009D008202062A068A1140843A0600D48C4
:105D0000C169491CC1612068C006C00F07D0E069A5
:105D1000C006C00F03D01020206200F085F9E069B2
:105D20004006C00F03D04020206200F0CDF910BD26
:105D300000440040FC030020F8B5614CE069800697
:105D4000C00F09D0A08C5F4AC1B21068FF2803D2EF
:105D50005D4B1954401C1060E06900250006C00F1F
:105D60008026002810D05949594A0868136898427B
:105D700005D30D6015602068B043206004E0554AEB
:105D8000125C401C08602285E0690007C00F06D045
:105D900008202062A068012109030843A060206850
:105DA000C006C00F07D0E069C006C00F03D01020A6
:105DB000206200F091F9E06940274006C00F0028FA
:105DC00002D0276200F094F9434CE0698006C00FCE
:105DD00009D0A08C414AC1B21068FF2803D2404BC1
:105DE0001954401C1060E0690006C00F10D03D49F6
:105DF0003D4B08681A68904205D30D601D6020680D
:105E0000B043206004E0394A125C401C08602285DF
:105E1000E0690007C00F01D0082020622068C0069A
:105E2000C00F07D0E069C006C00F03D01020206269
:105E300000F076F9E0694006C00F02D0276200F05A
:105E40007BF92B4CE0698006C00F09D0A08C294A51
:105E5000C1B210683F2803D2274B1954401C106070
:105E6000E0690006C00F10D02449254B08681A6865
:105E7000904205D30D601D602068B043206004E0AF
:105E8000204A125C401C08602285E0690007C00FB0
:105E900001D0082020622068C006C00F07D0E0694A
:105EA000C006C00F03D01020206200F05DF9E06949
:105EB0004006C00F02D0276200F062F9F8BD000072
:105EC0000048004070010020501B00209C01002071
:105ED00074010020901A002000500040780100203A
:105EE000501C0020A00100207C010020D01A0020BE
:105EF0000014014080010020501D0020A40100205A
:105F000084010020101B00200548416A491C4162A1
:105F100004490968002901DD0121C16770470000BB
:105F200068030020E4000020F8B5144D0C46064636
:105F300002212846FDF7F8FA10200090104B324657
:105F400002212846FDF7DAFA224602212846FDF70B
:105F50001DFB02212846FDF7F3FA0A4804630121DC
:105F6000417202212846FDF7F7FA05482838816872
:105F70008022114381602046F8BD000000000240ED
:105F800028380140680300200248016A491C016268
:105F9000704700006803002010B50A48407A0028C6
:105FA0000DD1084C206F5834002808D12046FBF74B
:105FB000EBFB0146E26820688018FFF7B5FF002080
:105FC00010BD000068030020F8B5144D0C460646CD
:105FD00005212846FDF7A8FA002000903346104A14
:105FE00005212846FDF78AFA224605212846FDF7B5
:105FF000CDFA05212846FDF7A3FA0A48446301219A
:10600000817205212846FDF7A7FA054824388168E2
:106010004022114381600020F8BD000000000240D2
:1060200024440040FC0300200A480B4900794058F2
:10603000802180B2081A0949012208600849CA670C
:106040004A6A521C4A62002803DD01200549000704
:10605000486070473071000804000240E8000020EA
:10606000FC03002000ED00E0F8B5144D0C46064698
:1060700004212846FDF758FA10200090104B3246B4
:1060800004212846FDF73AFA224604212846FDF766
:106090007DFA04212846FDF753FA0A4804630121DA
:1060A000417204212846FDF757FA054828388168CF
:1060B0008022114381602046F8BD000000000240AC
:1060C00028440040FC0300200248016A491C016288
:1060D00070470000FC03002003484068002802D0FD
:1060E00002490120C86770476C010020D4180020C5
:1060F0007047000010B50C460A4601460548FBF7FC
:1061000056F8054884600548016880221143016003
:1061100010BD0000901A00206C01002000480040D3
:106120000348C068002802D002490120C8677047B0
:106130006C010020681900207047000010B50C4663
:106140000A4601460548FBF732F805480461054850
:10615000016880221143016010BD0000D01A0020A8
:106160006C0100200050004003484069002802D024
:1061700002490120C86770476C010020FC1900200B
:106180007047000010B50C460A4601460548FBF76B
:106190000EF80548846105480168802211430160BA
:1061A00010BD0000101B00206C01002000140140F5
:1061B00010B5054C0A46638821465B1C4380FBF7FB
:1061C0003DFA002010BD0000007C00080B4610B511
:1061D000054944054118002C184602D000F066F825
:1061E00010BDFBF72BFA10BD001002080B46034947
:1061F00010B541181846FBF721FA10BD000002083F
:1062000070B50C460B494118002B08D00A4D4519B2
:10621000012B03D0094B9B8A002B00D12946400556
:10622000204603D000F042F8002070BDFBF706FACC
:10623000FAE700000080000800A00008B418002061
:10624000F8B54188174A491C4180154901807E21D3
:1062500000250A52ED43802300221146124C0026ED
:1062600059430C19314603E0675CFF2F04D1491CE8
:106270009942F9DB002E03D0521C082AEDDB00E026
:106280001546082D06D208495D436918802200F0A2
:106290000DF803E080220449FBF7D0F90020F8BD97
:1062A000AA550000A55A000000C00008F8B516461F
:1062B0000F460546FDF72AFA0024761C76080EE004
:1062C000600042195278295C120289188AB2C119F9
:1062D00000230220FDF7BEF9002802D0641CA6426C
:1062E000EED8054A1169802319431161002801D0B5
:1062F0000020F8BD0120F8BD00200240FEE70000AC
:106300000FB410B504A9074B02AA039800F028F8AF
:10631000044602A9002000F05DFA204610BC08BC2B
:1063200004B01847D567000830B47446641E257859
:10633000641CAB4200D21D46635D5B00E31830BCB9
:10634000184702E008C8121F08C1002AFAD1704796
:106350007047002001E001C1121F002AFBD17047E5
:10636000FFB591B00F460546002606E025280AD065
:10637000149A139990476D1C761C28780028F5D143
:10638000304615B0F0BD002400940121F34A029478
:1063900000E004436D1C2B780846203B98401042D7
:1063A000F7D128782A280ED0022128780246303AE0
:1063B000092A15D8009A0A235A43303A80180C4308
:1063C0006D1C0090F1E701CF0090002805DA012054
:1063D00040030443009840420090022004436D1C97
:1063E00028782E2815D10420044368786D1C2A28AB
:1063F0000AD101CF6D1C02900BE002990A22514391
:10640000303940186D1C029028780146303909292E
:10641000F3D928786C2810D006DC4C281AD06828CC
:106420000ED06A2817D104E0742813D07A2812D12C
:1064300010E00120400504430CE00121090501E0C2
:10644000032109050C436978814203D1012000052D
:1064500024186D1C6D1C287803906E281ED00CDC4F
:10646000632831D004DC00288AD0582811D1B2E04A
:1064700064287BD069280CD178E073282DD004DC07
:106480006F2870D0702804D1A7E075286CD07828C8
:106490006BD0149A13999047761C62E06002400F0B
:1064A000022807D003280AD0042838680AD00660DA
:1064B0003F1D56E03868F11706604160F8E738681C
:1064C0000680F5E70670F3E738786946087400201F
:1064D000487404A80390012003E03868039000206A
:1064E000C0433F1D61070FD5002101E00199491C00
:1064F000029A0191914213DA8142F7DB019A0399E2
:10650000895C0029F2D10BE0002101E00199491CCE
:1065100001918142FADB019A0399895C0029F5D146
:1065200001990098139A401A00902146149B00F09C
:106530003BF901998019461807E003980399007800
:10654000491C0391149A139990470198401E019099
:10655000401CF2D12146149B139A009800F014F9C4
:1065600086196D1C09E741E033E034E00A20002180
:10657000049005916002410F022905D001CFC21796
:106580009446032905D007E0FF1DFF08FF0003CF55
:1065900006E000B2C2179446042902D140B2C117E6
:1065A0008C4600226146944506DA0A4600214042A4
:1065B00091418C462D2102E0210504D52B216A460C
:1065C0001176012103E0E10701D02021F7E70191D5
:1065D00054E00A200BE0102009E010200490002174
:1065E0000420044308200591029003E008200021C4
:1065F000059104906002410F022905D001CF0022CD
:106600009446032906D006E0FF1DFF08FF0003CFD4
:106610008C4603E080B2042900D1C0B20021019170
:1066200021072BD50399702906D0049A1021059BC8
:106630004A401A4305D00EE040216A4611760121F6
:1066400008E06146014306D030216A46117603997D
:10665000517602210191049A0821059B4A401A4370
:106660000CD16146014301D1610707D530216A464B
:106670001176012101910299491E0291039958292D
:1066800004D037A103910FA90F910DE039A1F9E7CB
:106690006146059B049AFAF7B8FD039B8C469B5C08
:1066A0000F9A521E0F92137061460143F0D10F985A
:1066B00007A9081A20300390600704D501200004C0
:1066C0008443029801E0012002900399884201DD91
:1066D000401A00E000204118029001980918009823
:1066E000401A0090E00306D42146149B139A0098A8
:1066F00000F05AF886190020049008E006A9085C0A
:10670000149A139990470498401C761C04900199A0
:106710008842F3DBE0030CD52146149B139A0098C2
:1067200000F042F8861904E0149A3020139990473B
:10673000761C0299481E02900029F5DC08E00F98AB
:106740000F990078491C0F91149A13999047761C61
:106750000399481E03900029F1DCFBE6092801009B
:1067600030313233343536373839616263646566C7
:106770000000000030313233343536373839414289
:106780004344454600000000F8B5044600251E4677
:106790001746880404D405E039462020B0476D1C14
:1067A000641EF9D52846F8BDFFB50446002581B022
:1067B0001E46C80301D5302700E02027880404D5F1
:1067C00005E038460399B0476D1C641EF9D528468C
:1067D00005B0F0BD0A68531C0B60107070470000D4
:1067E00010B50A2101A0FEF70BFD10BD1B5B324A5C
:1067F0001B5B303B304800002D2110B5C90140180B
:1068000000F0DEFB10BD000030B503460B48002948
:1068100000D101210A4C491E0ED31A7850400022A3
:10682000C50702D04008604000E04008521CD2B2C8
:10683000082AF5D35B1CEEE730BD0000FFFF000027
:1068400001A0000070B50A4DFF23EE1D1A46F9366F
:1068500005E0047854402A5D5A40335D401C0C46E4
:10686000491E89B2002CF4D11802104370BD0000FB
:106870003673000870B504460C4800220C4E11E037
:106880002378521C1D4645402D07ED0E755B00090F
:106890004540180968400007C00E305A2B0958407F
:1068A00092B2641C8A42EBD370BD0000FFFF00006F
:1068B0006870000810B5084A084B07E00478544097
:1068C0002406E40D1C5B120A6240401C491EF5D2EE
:1068D000D04380B210BD0000FFFF000036710008F9
:1068E00006C00021016041608160C1600122026137
:1068F000416108467047000088B0002080F310888E
:10690000FE4F0125FF203D830530FD4BA022009066
:10691000991AFC48FBF70EFC4020FB4B0246191A63
:106920000090FA48FBF706FCFBF70CF8F84C002641
:10693000F8482667C06A6066F7480068A066F748AE
:10694000406AE066FFF706F9F649F5480860FBF78C
:1069500001FCFDF7E3F803200390049601A90596D6
:106960000295F148FCF7E8FEFDF7C4F8FCF73CFDA2
:10697000EE48FEF739FD3D83FEF732FDA063EC499A
:1069800060630D70EB4902070D70EB49120F0A703E
:10699000EA49EB4F1F2804D0C00605D50D703E70A4
:1069A00004E0E8480570F9E70E703D70E6480278AB
:1069B000E24801780220FBF70DFDE4490220FBF7D5
:1069C00081FFDD48E04900780870E1490120087046
:1069D000E120E04940020860FDF738F9FDF7C8F909
:1069E000FDF786FADC48006820210843DA49086090
:1069F0000868102528430860FDF7C4FAD7480068E6
:106A000020210843D5490860086828430860FDF73D
:106A100003FBD34801682022114301600168294328
:106A20000160FDF715F8FDF7CDF8FDF7E5F8CD4865
:106A30000168012211430160CB4801682022114303
:106A4000016001682943016001684022114301602F
:106A50008021C648FFF7B8FAC5480168294301609C
:106A600001684022114301600A20FAF74FFF01201C
:106A7000FEF7BEFE0020FEF7A5FE0020FEF7BCFBE1
:106A80000120FAF7D1FD0020FEF7A8FEFEF720FF57
:106A9000FAF726FF6066994D002028826882A34895
:106AA000C0882882288A01280AD1FBF7FDFA208FA6
:106AB000202108406882688A002801D0FEF7CAFFBA
:106AC000AC4E5A2070840020C043FDF7C5FE1B2148
:106AD000A948890145180F21C90140180090A74F06
:106AE0000020387001207870FAF7FAFE3861FAF762
:106AF0001BFF0790FEF774FC07468048008AC0071A
:106B00000BD0B806208F04D5800606D4FEF7A2FF6E
:106B100003E0800601D5FEF7D5FFA7630798E06381
:106B20000920C0060069009988847F480069C884EC
:106B3000934800690885934800694885FAF75EFE26
:106B40003075FAF7CDFE8D4F78618F4800680028C8
:106B500001D00020B082206CC006C00E02281CD1DB
:106B6000FAF7C4FB8848016800290ED00021B182E1
:106B700086490A68002A10D10068086084480068C5
:106B800084490860FDF7D0FE07E080490A68002AC2
:106B900003D000680860FDF7DFFE5848008A01282E
:106BA0000BD15648818A002927D07B49B960C18A18
:106BB0007A480160B868FDF7D7FE606E7969616652
:106BC000081AA066E16E884200D2E066216F884212
:106BD00000D92067FAF784FEB86158480078002889
:106BE00006D059480078002802D00220FBF778FC34
:106BF0000798800403D5012002E06949D6E7002008
:106C000038700798000501D5012000E00020787059
:106C10004B48007800281AD00220FBF7A3FE606CD6
:106C2000002801D15F4908845E485F49008C888252
:106C30005E490868800401D5012000E0002038701A
:106C40000868000501D5012000E000207870554853
:106C5000B18A0180018CB186F18A4180318B8180BB
:106C6000718BC180606C002801D0401E6064A06CF4
:106C7000002801D0401EA0642048018B00293BD091
:106C80007878FEF7B5FD7878FEF79CFD7878FEF70A
:106C90008DFD7878002801D1012000E00020FEF76A
:106CA0009DFDFAF71DFEF861FAF71AFE3862FAF751
:106CB00017FE0A2178620846FAF708FA0020401CFD
:106CC0004028FCDB206C401C20640E48C06F00286C
:106CD00013D037480268002A0FDD3648007825288F
:106CE0006AD092B233490120FDF7FEF90549002030
:106CF000C8672F49086098E05FE083E0B41800207F
:106D0000301E002068030020741F0020FC030020B8
:106D10008016002080F7FF1FD800002000100240DE
:106D200010270000A8010020000400488010002067
:106D3000D4010020D5010020F0000020EC0000204C
:106D4000ED00002020010020F7000020992200081B
:106D5000F1000020DC00002000480040005000400E
:106D600000140140001000400038014010050020D0
:106D7000004400404013002000110020AC0100201E
:106D800000080048000C0048600100206401002059
:106D9000880100206801002000A0000838010020C0
:106DA00000800008280C002000150020240100208D
:106DB000E4000020900400201FE0008A01280FD08A
:106DC000606C002810D07878FEF712FDA06C0028C7
:106DD0000CD07878FEF7F6FC7878FEF7E7FC5DE7F4
:106DE000554800680028EFD03878EDE70020FEF71E
:106DF000E9FC0020FEF7DAFC4EE750490120FBF7E2
:106E00001BFF73E74E49786888420DD94D484168A9
:106E100001221205114341604168520003235B05C2
:106E200099431143416001E0401C78604648007876
:106E3000002802D00020FAF769FD444FF86F0028BF
:106E400008D0434801784348FEF794FB40490020AE
:106E50000860F86740484149407D0870FEF74AFBEA
:106E60003F48007870753F48C06F00280CD0A88854
:106E70003D4F401CA8803D4900203A68FDF714FBB7
:106E8000002038493860C86739480088E8803948A8
:106E90000088288138480088688138480088A8819F
:106EA00037480088E8813748C06F00280CD0A88A8E
:106EB000354F401CA882354901203A68FDF7F4FAA5
:106EC000002030493860C86731483A4B0088E88272
:106ED0003048008828833048008868832F4800881D
:106EE000A88486462E480088E88484462D48018878
:106EF0002D482985008868852C480088A8852C485D
:106F00000288AA868288EA8602892A8782896A8715
:106F1000028AAA87828AEA87028B1A80808B58802D
:106F20007046F082604630837183B08EFEF764F95C
:106F3000224921480860D2E5780E00209004002004
:106F4000C027090000380140ED000020FC19002096
:106F500080010020501D002060130020D601002079
:106F6000D7010020D418002070010020501B002001
:106F7000040200200C020020140200203402002031
:106F80003C0200206819002078010020501C0020DD
:106F90000802002010020020180200203802002001
:106FA00024020020280200202C02002030020020B1
:106FB000B41F002000180020AAAA000000300040E2
:106FC0002D2110B54902002800DA4018FAF7A4F87C
:106FD000C817800E4018821180098001081A1C4BC6
:106FE00040245A2A04DA91005A58C918496808E01E
:106FF000B42A0FDAB421891A89005A58C91880397D
:10700000C96F231A534348431818C117890E08182B
:10701000801110BDFF210F318A4206DA0D4992001E
:1070200051185A58C918496807E0FF216931891A6F
:1070300089005A58C9188039C96F231A53434843E5
:107040001818C117890E08188011404210BD0000A1
:107050004075000830FDFFFF1122334455667788E4
:1070600099AABBCCDDEEFF00000001CC01D80014D2
:1070700001F0003C002801E401A0006C007801B49C
:107080000050019C01880044011109010201040122
:1070900004010000000000000000000000000600E5
:1070A000AA550000000100000000000001000100DE
:1070B00000090000000000000000020000000009BC
:1070C00000000000000000000000000000000000C0
:1070D0000000000000000000101010101010101030
:1070E0001010101010101010100020003000400080
:1070F00050006000030000000400000005000000D4
:107100000600000007000000080000000900000061
:107110000A0000000B0000000C0000001100A55A3E
:10712000AA55000000000000000000000000000060
:10713000081C304458000000891112239B32244659
:10714000AD573665BF74488CC19D5AAFD3BE6CCA6B
:10715000E5DB7EE9F7F88110080193331A22A55682
:107160002C47B7753E64C99C408DDBBF52AEEDDA4B
:1071700064CBFFF976E802218B3010029913266761
:10718000AF763444BD554AADC3BC588ED19F6EEB2B
:10719000E7FA7CC8F5D983310A2091121803A77742
:1071A0002E66B5543C45CBBD42ACD99E508FEFFB0B
:1071B00066EAFDD874C904428D5316619F7020049D
:1071C000A9153227BB364CCEC5DF5EEDD7FC6888EB
:1071D000E1997AABF3BA85520C4397711E60A11402
:1071E0002805B3373A26CDDE44CFDFFD56ECE998CB
:1071F0006089FBBB72AA06638F7214409D512225E1
:10720000AB343006B9174EEFC7FE5CCCD5DD6AA9AA
:10721000E3B8788AF19B87730E6295501C41A335C1
:107220002A24B1163807CFFF46EEDDDC54CDEBB98A
:1072300062A8F99A708B088481951AA793B62CC21C
:10724000A5D33EE1B7F04008C919522BDB3A644E92
:10725000ED5F766DFF7C899400859BB712A6ADD259
:1072600024C3BFF136E0C1184809D33B5A2AE55E72
:107270006C4FF77D7E6C0AA583B4188691972EE338
:10728000A7F23CC0B5D14229CB38500AD91B666F52
:10729000EF7E744CFD5D8BB502A499961087AFF319
:1072A00026E2BDD034C1C3394A28D11A580BE77F32
:1072B0006E6EF55C7C4D0CC685D71EE597F4288074
:1072C000A1913AA3B3B2444ACD5B5669DF78600C12
:1072D000E91D722FFB3E8DD604C79FF516E4A990D9
:1072E0002081BBB332A2C55A4C4BD7795E68E11CF2
:1072F000680DF33F7A2E0EE787F61CC495D52AA1B8
:10730000A3B03882B193466BCF7A5448DD59622DD1
:10731000EB3C700EF91F8FF706E69DD414C5ABB198
:1073200022A0B9923083C77B4E6AD5585C49E33DB1
:107330006A2CF11E780F00C1814001C0804101C05C
:10734000804100C1814001C0804100C1814000C135
:10735000814001C0804101C0804100C1814000C125
:10736000814001C0804100C1814001C0804101C015
:10737000804100C1814001C0804100C1814000C105
:10738000814001C0804100C1814001C0804101C0F5
:10739000804100C1814000C1814001C0804101C0E5
:1073A000804100C1814001C0804100C1814000C1D5
:1073B000814001C0804101C0804100C1814000C1C5
:1073C000814001C0804100C1814001C0804101C0B5
:1073D000804100C1814000C1814001C0804101C0A5
:1073E000804100C1814001C0804100C1814000C195
:1073F000814001C0804100C1814001C0804101C085
:10740000804100C1814001C0804100C1814000C174
:10741000814001C0804101C0804100C1814000C164
:10742000814001C0804100C1814001C0804101C054
:10743000804100C1814000C0C101C30302C2C60631
:1074400007C705C5C404CC0C0DCD0FCFCE0E0ACA9C
:10745000CB0BC90908C8D81819D91BDBDA1A1EDEEC
:10746000DF1FDD1D1CDC14D4D515D71716D6D2129C
:1074700013D311D1D010F03031F133F3F23236F6AC
:10748000F737F53534F43CFCFD3DFF3F3EFEFA3A5C
:107490003BFB39F9F83828E8E929EB2B2AEAEE2EEC
:1074A0002FEF2DEDEC2CE42425E527E7E62622E25C
:1074B000E323E12120E0A06061A163A3A26266A6AC
:1074C000A767A56564A46CACAD6DAF6F6EAEAA6A1C
:1074D0006BAB69A9A86878B8B979BB7B7ABABE7E6C
:1074E0007FBF7DBDBC7CB47475B577B7B67672B21C
:1074F000B373B17170B050909151935352929656AC
:107500005797559594549C5C5D9D5F9F9E5E5A9ADB
:107510009B5B99595898884849894B8B8A4A4E8E6B
:107520008F4F8D4D4C8C44848545874746868242DB
:10753000438341818040081C304458081C30445823
:1075400000000000110000002300000034000000D3
:107550004600000057000000690000007A000000AB
:107560008B0000009C000000AE000000BF00000087
:10757000D0000000E1000000F20000000301000064
:107580001401000024010000350100004601000044
:10759000560100006601000077010000870100002D
:1075A00097010000A7010000B6010000C60100001D
:1075B000D5010000E5010000F40100000302000015
:1075C00012020000210200002F0200003E02000013
:1075D0004C0200005A020000680200007502000020
:1075E00083020000900200009D020000AA02000039
:1075F000B7020000C3020000CF020000DB0200005F
:10760000E7020000F3020000FE0200000903000090
:10761000140300001F0300002903000033030000CF
:107620003D03000047030000500300005903000021
:10763000620300006B030000730300007B03000083
:10764000830300008A0300009203000099030000F6
:107650009F030000A6030000AC030000B20300007B
:10766000B7030000BC030000C1030000C603000014
:10767000CA030000CE030000D2030000D6030000BE
:10768000D9030000DC030000DE030000E10300007A
:10769000E3030000E4030000E6030000E70300004A
:1076A000E7030000E8030000E8030000E80300002F
:1076B000E7030000E7030000E6030000E403000026
:1076C000E3030000E1030000DE030000DC03000030
:1076D000D9030000D6030000D2030000CE0300004F
:1076E000CA030000C6030000C1030000BC03000081
:1076F000B7030000B2030000AC030000A6030000C3
:107700009F03000099030000920300008A03000019
:10771000830300007B030000730300006B03000081
:1077200062030000590300005003000047030000FB
:107730003D03000033030000290300001F03000085
:107740001403000009030000FE020000F302000021
:10775000E7020000DB020000CF020000C3020000CD
:10776000B7020000AA0200009D0200009002000083
:107770008302000075020000680200005A02000047
:107780004C0200003E0200002F0200002102000017
:107790001202000003020000F4010000E5010000F5
:1077A000D5010000C6010000B6010000A7010000DD
:1077B00097010000870100007701000066010000CA
:1077C00056010000460100003501000024010000C0
:1077D0001401000003010000F2000000E1000000BD
:1077E000D0000000BF000000AE0000009C000000C0
:1077F0008B0000007A0000006900000057000000C4
:1078000046000000340000002300000011000000CA
:1078100000000000EFFFFFFFDDFFFFFFCCFFFFFFD9
:10782000BAFFFFFFA9FFFFFF97FFFFFF86FFFFFFE4
:1078300075FFFFFF64FFFFFF52FFFFFF41FFFFFFE8
:1078400030FFFFFF1FFFFFFF0EFFFFFFFDFEFFFFEB
:10785000ECFEFFFFDCFEFFFFCBFEFFFFBAFEFFFFEB
:10786000AAFEFFFF9AFEFFFF89FEFFFF79FEFFFFE2
:1078700069FEFFFF59FEFFFF4AFEFFFF3AFEFFFFD2
:107880002BFEFFFF1BFEFFFF0CFEFFFFFDFDFFFFBA
:10789000EEFDFFFFDFFDFFFFD1FDFFFFC2FDFFFF9C
:1078A000B4FDFFFFA6FDFFFF98FDFFFF8BFDFFFF6F
:1078B0007DFDFFFF70FDFFFF63FDFFFF56FDFFFF36
:1078C00049FDFFFF3DFDFFFF31FDFFFF25FDFFFFF0
:1078D00019FDFFFF0DFDFFFF02FDFFFFF7FCFFFF9E
:1078E000ECFCFFFFE1FCFFFFD7FCFFFFCDFCFFFF3F
:1078F000C3FCFFFFB9FCFFFFB0FCFFFFA7FCFFFFCD
:107900009EFCFFFF95FCFFFF8DFCFFFF85FCFFFF4A
:107910007DFCFFFF76FCFFFF6EFCFFFF67FCFFFFB7
:1079200061FCFFFF5AFCFFFF54FCFFFF4EFCFFFF12
:1079300049FCFFFF44FCFFFF3FFCFFFF3AFCFFFF59
:1079400036FCFFFF32FCFFFF2EFCFFFF2AFCFFFF8F
:1079500027FCFFFF24FCFFFF22FCFFFF1FFCFFFFB3
:107960001DFCFFFF1CFCFFFF1AFCFFFF19FCFFFFC3
:1079700019FCFFFF18FCFFFF18FCFFFF18FCFFFFBE
:1079800019FCFFFF19FCFFFF1AFCFFFF1CFCFFFFA7
:107990001DFCFFFF1FFCFFFF22FCFFFF24FCFFFF7D
:1079A00027FCFFFF2AFCFFFF2EFCFFFF32FCFFFF3E
:1079B00036FCFFFF3AFCFFFF3FFCFFFF44FCFFFFEC
:1079C00049FCFFFF4EFCFFFF54FCFFFF5AFCFFFF8A
:1079D00061FCFFFF67FCFFFF6EFCFFFF76FCFFFF13
:1079E0007DFCFFFF85FCFFFF8DFCFFFF95FCFFFF8B
:1079F0009EFCFFFFA7FCFFFFB0FCFFFFB9FCFFFFF1
:107A0000C3FCFFFFCDFCFFFFD7FCFFFFE1FCFFFF46
:107A1000ECFCFFFFF7FCFFFF02FDFFFF0DFDFFFF8A
:107A200019FDFFFF25FDFFFF31FDFFFF3DFDFFFFBE
:107A300049FDFFFF56FDFFFF63FDFFFF70FDFFFFE8
:107A40007DFDFFFF8BFDFFFF98FDFFFFA6FDFFFF04
:107A5000B4FDFFFFC2FDFFFFD1FDFFFFDFFDFFFF14
:107A6000EEFDFFFFFDFDFFFF0CFEFFFF1BFEFFFF16
:107A70002BFEFFFF3AFEFFFF4AFEFFFF59FEFFFF0E
:107A800069FEFFFF79FEFFFF89FEFFFF9AFEFFFF01
:107A9000AAFEFFFFBAFEFFFFCBFEFFFFDCFEFFFFEB
:107AA000ECFEFFFFFDFEFFFF0EFFFFFF1FFFFFFFCE
:107AB00030FFFFFF41FFFFFF52FFFFFF64FFFFFFAB
:107AC00075FFFFFF86FFFFFF97FFFFFFA9FFFFFF87
:107AD000BAFFFFFFCCFFFFFFDDFFFFFFEFFFFFFF60
:107AE000000000000000000001020304060708096E
:107AF0000000000001020304187B0008C000002001
:107B000088010000B0120008487B000848020020ED
:107B1000704700005263000801159201C7C20100BE
:107B200040420F52010433010101C2014201429758
:107B30000569FFFFFFFFC3102704478000080540C9
:087B4000A560A565631BB700F9
:04000005080010B926
:00000001FF
